:1000000000308A00C62C00008A1D0A128A190A16BE
:100010008A11831A0F28A500030EA6001428831244
:10002000A500030EA600A6140A08AD00A50E04083C
:10003000A7002008A8002108A9002208AA00230878
:10004000AB002408AC0083128B1E28280B1946280D
:100050008C308400801E2E288C1A482827088400A3
:100060002808A0002908A1002A08A2002B08A30044
:100070002C08A4002D088A000A1A8A150A12260ED6
:1000800083008312250EA618831609008A11FE2804
:100090008A1185290A108A100A1182077434723471
:1000A0006134663466346934633400340A108A106B
:1000B0000A118207423461346434203443345234A8
:1000C000433400340A108A100A1182074234613422
:1000D000643420346C3465346E346734743468347A
:1000E00000340A108A100A118207003410342034B8
:1000F0003034403450346034703481349134A1341D
:10010000B134C134D134E134F1340A108A100A1107
:10011000820700342134423463348434A534C63435
:10012000E734083429344A346B348C34AD34CE345B
:10013000EF340A108A100A11820730343134323415
:100140003334343435343634373438343934413454
:100150004234433444344534463400340A108A105F
:100160000A118207533465346E34643469346E3452
:10017000673420346D3465347334733461346734D8
:10018000653400340A108A100A1182074734453456
:1001900054342034443441345434413420345034C1
:1001A0004B34543400340A108A100A118207503438
:1001B0004F344C344C34203450344B3454340034A9
:1001C0000A108A100A11820743344D3444343A34F9
:1001D000203400340A108A100A118207573461341F
:1001E0006934743469346E3467342E342E342E34CA
:1001F0002E342E342E342E342E340034FF30031798
:10020000810003130B110B118A112E283608A43C10
:10021000031D0E290130A100112911290030A10070
:10022000112900343108A00003193F2901302002B0
:10023000031946290230200203194A2903302002FB
:1002400003194E290430200203195C2905302002CD
:100250000319682906302002031973290730200288
:10026000031977290830200203197C29093020025C
:1002700003197D29FF30200203197E297F293008C8
:10028000B2003008023C0319B10A81293008B300DA
:10029000B10A81293008B400B10A81293008B500BB
:1002A0003508403C03185929FF30B1000130FC00EB
:1002B0005B29FB01B10A81293008B6000621A1089B
:1002C000031965290530B10067290630B10081297D
:1002D00037307B07840030088000FB0A35087B023A
:1002E0000319B10A81293008F700B10A81293008C1
:1002F000F8000830B1008129812981298129B101C3
:1003000081293108A1008A1193298C1E9D29FF3073
:100310000317810003131A08B00018080639003AC1
:10032000031D9529122918169B2918121A08B000C6
:100330001A08B00018168C1285298C128A112E28E2
:10034000BC30840000080319B4290130A100A001C9
:10035000A00BA829A10BA7294A30A000A00BAE2909
:1003600000000000800BA529003402308316BC0079
:100370008312A021003401308316BC008312A02117
:1003800083163208831286008515B5218511B521A3
:10039000003483163A08BB00831205118316220825
:1003A0000139003A0319D6298312D929831205107D
:1003B000DA290514851183163A08831286008515FB
:1003C000B521851183163B08BA00BA0EF030BA0584
:1003D00083120511831622080139003A0319F22904
:1003E0008312F52983120510F62905148511831649
:1003F0003A08831286008515B5218511B521003490
:1004000084308316810083128B01073083169F008E
:10041000850186010F30870088018901FF30831232
:1004200087008316A2012830B2008312BB21053059
:100430008316BC008312A02128308316B2008312D9
:10044000BB2101308316BC008312A0212830831603
:10045000B2008312BB2101308316BC008312A0219D
:1004600028308316BA008312C9210C308316BA00D3
:100470008312C92101308316BA008312C9210630C4
:100480008316BA008312C92180308316BA00831202
:10049000C92101308316A2008312981718138316FE
:1004A0001813193099001815181298168312181677
:1004B0000B17F73087008A11242D83163208831218
:1004C000AE00831633088312AF00B1018712831682
:1004D0008C1683120034831622108312B521003447
:1004E000831622148312B52100346B22C030831688
:1004F000BA008312C9217022003475228316A30129
:100500008312831623080F3C0318882A8312922A29
:10051000831220308316BA008312C9218316A30ADE
:100520008312812A752200348316370883129900BA
:10053000831618080239003A031DA02A8312982A4C
:100540008312A22A0034790E8316BA000F30BA053E
:100550003908BA068312790E8316BB00F030BB054A
:1005600083127A0EA0000F30A005200883163B04EA
:100570008312F900FA0EF030FA0583163A08831256
:100580007120A100F90683163A0883128520A10084
:10059000FA0600348316370EB8000F30B805380855
:1005A000B9008312A322831637080F39B800B900A7
:1005B0008312A322003483168C1283128716013013
:1005C0008316BC008312A021FF30F900FA008316C5
:1005D000B501831283163508023C0318F12A8312F1
:1005E000FA2A83128316B701831294228316B50A5E
:1005F0008312EA2A02308316B7008312CA2202301D
:100600008316B700831294222E088316B700831234
:10061000CA222E088316B700831294222F0883164D
:10062000B7008312CA222F088316B70083129422C0
:1006300083163308B7008312CA2283163308B70023
:100640008312942283163208B7008312CA228316BB
:100650003208B700831294228316B308031D322B8D
:100660008312652B83128316B50183128316330818
:100670003502031C3D2B83124C2B83128316340846
:10068000350784000008B6003608B7008312CA2276
:100690008316B50A8312362B8316B501831283168F
:1006A00033083502031C562B8312652B83128316E5
:1006B0003408350784000008B6003608B7008312F6
:1006C00094228316B50A83124F2B79088316B7003C
:1006D000831294227A088316B70083129422013081
:1006E0008316BC008312A021871283168C168312F6
:1006F00000348316360E8312A0000F30A0052008A8
:100700000F3999208316B900BA008312C9218316C4
:1007100036080F39831299208316B800BA00831265
:10072000C92100348316B201B30183120B138B135A
:100730008B1B972B3108083C031D852C2E08330298
:10074000031DAC2BA32B2F083402031DAC2B01304F
:100750008316B2008312C22B7D228316B40183124A
:100760008316340883124A2000380319BD2B8316E0
:10077000B40ABA008312C921B02BC8308316BC005A
:100780008312A021FF30F900FA0002308316B7006F
:100790008312CA2233088316B7008312CA22340890
:1007A0008316B7008312CA2235088316B700831256
:1007B000CA2236088316B7008312CA220621A1086E
:1007C0000319FA2B8316B4018312350883163402F9
:1007D000031CEC2B8312FA2B831237308316340759
:1007E00084000008B500B7008312CA228316B40A39
:1007F0008312E52B79087702031D062CFF2B7A085C
:100800007802031D062C0930B100382C0230FC00A0
:10081000FF30B1007D2277088316B600831279235A
:1008200078088316B6008312792320308316BA0025
:100830008312C92179088316B600831279237908B7
:100840008316B60083127923FF308316BC0083120F
:10085000A021FF308316BC008312A021FF30831635
:10086000BC008312A021FF308316BC008312A0219C
:100870003108A1002108B100310F3F2C432C310871
:10088000093C031D852C310F742C7D227C08023C11
:10089000031D5B2C8316B401831283163408831264
:1008A0005620003803195A2C8316B40ABA00831252
:1008B000C9214D2C6D2C7C0B6D2C8316B401831239
:1008C0008316340883126220003803196D2C8316B6
:1008D000B40ABA008312C921602CC8308316BC0048
:1008E0008312A021B101852C3108093C031D852C00
:1008F0008316B208031D7E2C8312842C83120130D0
:100900008316B3008312852CB101C0308B0483168B
:1009100033088312A1008A11D22D83163208840075
:10092000831236088000831633088400831235084A
:1009300080008316B5018312350883163502031C27
:10094000A32C8312B62C8312831634083507B60005
:100950003730350784000008B700360884003708B0
:10096000800083128316B50A83129C2C83163408E8
:1009700083123507840080018A11E42D6B228030B8
:100980008316BA008312C9217022003484011F30FB
:1009900083059F30840007308000AE01AF01B001B5
:1009A000B101B201B301B401B501B601B701B8019B
:1009B000B901BA01BB01BC01BD01BE01BF01C0014B
:1009C000C101C201C301C401C501C601C701C801FB
:1009D000C901CA01CB01CC01CD01CE01CF01D001AB
:1009E000D101D201D301D401D501D601D701D8015B
:1009F000D901DA01DB01DC01DD01DE01DF01E0010B
:100A0000E101E201E301E401E501E601E701E801BA
:100A1000E901EA01EB01EC01ED01EE01EF01F0016A
:100A2000F101F201F301F401F501F601F701F8011A
:100A3000F901FA01FB01FC01FD01FE01FF01831632
:100A4000A001A1018312002A8B128316B201831226
:100A5000831632088312AE2000380319352D831611
:100A6000B20ABA008312C921282D1030AE00AF009F
:100A70002E088316B20083122F088316B300831248
:100A80005D2248308316A4006530A5006C30A600B6
:100A9000A7006F30A800A90183127D228316B2013E
:100AA0008312831632088312C220003803195E2D88
:100AB0008316B20ABA008312C921512DA4308316BD
:100AC000B2000530B300A430B4008312DB22FA3048
:100AD0008316BC008312A021FA308316BC00831257
:100AE000A021FA308316BC008312A021FA308316AD
:100AF000BC008312A0217D228316B20183128316CB
:100B000032088312D320003803198C2D8316B20AC1
:100B1000BA008312C9217F2DA1308316B200B30120
:100B2000A430B4008312DB22FA308316BC00831297
:100B3000A021FA308316BC008312A021FA3083165C
:100B4000BC008312A021FA308316BC008312A021BE
:100B50001030AE001830AF002E088316B20083129A
:100B60002F088316B30083125D22A1308316B200D2
:100B7000B301A430B4008312DB22FA308316BC0028
:100B80008312A021FA308316BC008312A021FA3010
:100B90008316BC008312A021FA308316BC00831296
:100BA000A021922B21088316AE00AE08031DDA2D7A
:100BB0008312522E8312B0308316B200AF30B300CE
:100BC000A430B40083128D2C7D228316B2018312CF
:100BD000831632088312E02000380319F52D83169E
:100BE000B20ABA008312C921E82D83163008B60074
:100BF0008312792320308316BA008312C921831609
:100C0000AF08031D052E83121E2E83128316B10119
:100C1000831283162F083102031C102E83121E2EFE
:100C20008312A4308316310784000008B200BA0092
:100C30008312C9218316B10A8312092EFF3083164D
:100C4000BC008312A0212E088316B20083122F0845
:100C50008316B30083125D22BE248316A301831280
:100C6000831623080F3C0318372E8312412E83125C
:100C700020308316BA008312C9218316A30A831277
:100C8000302EBE248316B2018312831632088312DB
:100C9000EA2000380319522E8316B20ABA008312D2
:080CA000C921452E352D63002A
:02400E00723D01
:00000001FF
